:030000000219FDE5
:03000B000200AA46
:03002B0002015F70
:03005B000202F5A9
:030073000202DBAB
:1000800002030406080C10182030406080040608A3
:100090000C10182030406080A0C000070F1F3F0DDB
:1000A0000D0403060D0502030202C2AFC0D0C0E07A
:1000B000206217E5256002E473E525F4F58A758B67
:1000C00000D262D0E0D0D0D2AF3285268AC262E5BB
:1000D00026F4602F758B00D0E0D0D0C293C297C2B7
:1000E00095D2AF32C293C297C295206E0C2066099A
:1000F000740ED5E0FDE57E4290758B00D0E0D0D047
:10010000D2AF32758A00C28DD26201F901B930686E
:1001100005206602D29301B9306805206602D297A5
:1001200001B9306805206602D29501B9C2923068E3
:100130000A206607740CD5E0FDD29301B9C296304F
:10014000680A206607740CD5E0FDD29701B9C29405
:1001500030680A206607740CD5E0FDD29501B9C25B
:10016000AFC2AD53E6EFC0D0C0E0D2D3D2AFC2CE63
:10017000E52A6007207449152A21C07800790020FB
:10018000742EE580307E01F430E50278FF53DACF3B
:10019000207E0343DA20307E0343DA10C2D8C271D6
:1001A000E580307E01F430E50279FFC3E89970CB39
:1001B000306103752A40207403752A40885FD2702D
:1001C00020740DE52B6004152B21D043DA01C2D831
:1001D00020700221E3A85F206102C2702074022116
:1001E000E188227882B60403852224C3E525944061
:1001F0004002D26420CF0AD0E0D0D043E610D2AD86
:1002000032C2CF053A7802E52A6005307402152A19
:10021000C3E55F94014005756200412D756300756B
:100220006C00E5622401F56250037562FF7982B7C4
:10023000020D306D1DC3E52294324016854D2279A2
:1002400082B7030E306D0BC3E52294324004798EE1
:100250008722C3E5239522600840041523416105E8
:1002600023D8CA056CE56C7002156CD56D63756D8D
:10027000017805C3E56C956E4057C3E56C956F50EA
:10028000087801756D03020295C3E56C9570500501
:100290007801756D01C3E5659524401E7982B70428
:1002A0000241C6206D14852465E56C046003856EEB
:1002B0006C756D0175233C0202D1E565285005750A
:1002C00065FF41C6F565E5650470067563FF756CED
:1002D000FFD0E0D0D043E610D2AD32C2AFC0D05391
:1002E000E67FC26075910085569485579575910497
:1002F000D0D0D2AF32C2AF53E6EFC2ADC0D0C0E073
:10030000C0F0D2D3D2AFA8FBA9FCC2D83071026131
:100310005C53DACF207E0343DA10307E0343DA20C9
:10032000D271E580307E01F420E5026133882789AF
:1003300028A14153DACF207E0343DA20307E0343E5
:10034000DA10C2D8C271307402A12D7800E5803075
:100350007E01F430E502A12D885FA11553DACF208C
:100360007E0343DA20307E0343DA10C2712061023B
:10037000813553DACF207E0343DA10307E0343DA2F
:1003800020C2D8D271885A895BC3E89558F8E9959C
:1003900059F97B007E087A00C3E8948CE9940050F8
:1003A00005755E008127882178A2E6A8216055C3E3
:1003B000E894C8E994005008E4D2E4FB7A0A810288
:1003C000C3E89468E994015008E4D2E3FB7A0F8112
:1003D00002C3E894D0E994025008E4D2E2FB7A1E0A
:1003E0008102C3E894A0E994055008E4D2E1FB7AC5
:1003F0003C8102C3E89498E994085008E4D2E0FBF9
:100400007A787E00C3E8955CFCE9955DFD30E70AEB
:10041000ECF42401FCEDF43400FD755E00C3EC9AAD
:10042000ED9E5003755E01885C895D855A58855B39
:10043000597802A115C3E89527F8E99528F9307C89
:100440000281F9307B0281F9307A0281F220750253
:100450008158E9FDE8FC8177E9C313F9E813F83026
:10046000790281F2E9C313F9E813F830780281F2D6
:0F047000E9C313FDE813FC20612CC3EC941CEDD1
:10047F0094024002818EED701EC3EC94C850180593
:10048F0029E52970021529C3E529940A5002A12DE7
:10049F00755F00D270A12DE5296002152974002027
:1004AF007F037896E624FAFEE43400FFC3EC9EFC4B
:1004BF00ED9FFD50067800790081F9C3EC94FFEDB4
:1004CF009400400678FF790081F9EC8575F0A4C59A
:1004DF00F0A2F733F87900400302051578FF790091
:1004EF00020515E9C313F9E813F8307C0EE9600231
:1004FF0078FFC3E81338F8E43400F9C3E894FFE950
:10050F009400400278FF885FD270206102A12D74A1
:10051F001FF4552F4BF52FC274EB7002D274752A4E
:10052F0040307403752A0A306102A14120740353CD
:10053F00DAFE207403752B20D0F0D0E0D0D0D2ADEE
:10054F0043E6103279010205717903020571790AC8
:10055F00020571791E020571796402057179C8026D
:10056F0005717817E4D5E0FDD8FAD9F6227A147B15
:10057F00780205987A107B8C0205987A0D7BB4026D
:10058F0005987A0B7BC80205987902B27DE4C29672
:10059F00D5E0FDD297D5E0FDC297D5E0FDD296D537
:1005AF00E0FDD293E576D5E0FDC2937496D5E0FDDC
:1005BF00D9D9EAF8D5E0FDD8FBDBCEC29622C37CB1
:1005CF00007D0075F00005F0EA33FAEB33FB50F6CF
:1005DF00EB13FBEA13FAC3E9FFE8FEE89AF8E99B8D
:1005EF00F95004EFF9EEF8B3EC33FCED33FDD5F031
:1005FF00DFEDF9ECF822E889F08A20D2D4F8A9F0DF
:10060F007B0030F70B7BFFF42401F8E9F43400F999
:10061F00E88520F0A4ADF0F8E98520F0A4AFF0FE56
:10062F00ED2EF974003FFA7C04C3EA13FAE913F9CB
:10063F00E813F8DCF48BF030F70AE8F42401F8E95A
:10064F00F43400F9E889F0C2D4F8A9F0227882B620
:10065F0004030206FBC3E55F9419401EE52D540603
:10066F007018206D3678057994E7146007780A14AE
:10067F0060027812C3E54198401F306D09856765A8
:10068F00756CFF756D01852224E4F545F546F54738
:10069F00F548F549C26D0206FBD26D7994E71470E7
:1006AF0013E523F43333F913F8E9540104F9E8544B
:1006BF00FE0206EFE714147014E523F4333333F915
:1006CF0013F8E9540304F9E854FC0206F7E523F4A0
:1006DF0033333333F913F8E954070404F9E854F8C2
:1006EF00C39440F8E99400F98845894622C3E5414F
:1006FF0013F9E54013F8C3E54598F8E54699F95025
:10070F000CC3E89480E994FF4016020733C3E894C2
:10071F007FE994005003020733787F790002073393
:10072F00788079FF884A894B22E54A2547F8E54BBF
:10073F003548F9854B20E4300701F43549FA30E7A5
:10074F0009C3EA94F04015020771C3EA940F5003EE
:10075F0002077178FF79FF7A0F020771780079002D
:10076F007AF0C3E5249564500AC374019524500BA5
:10077F0002078FE54B20E70E02078FE54B30E706A8
:10078F00884789488A492278A4E6FAC3E54A33F8AC
:10079F00E54B33F9D105E930E70BC3E89480E994D1
:1007AF00FF4013E1C9C3E8947FE994005002E1C907
:1007BF00787F7900E1C9788079FFE820E715C3E5F4
:1007CF002398F84009C3E8940140030207F0780129
:1007DF000207F0E8F424012523F840030207F0781C
:1007EF00FF884C2278A5E6FAA848A949D105E93037
:1007FF00E70CC3E89401E994FF4016020824C3E80C
:10080F0094FFE99400500302082478FF790002084E
:10081F0024780179FFE920E715C3E54C98F84009E2
:10082F00C3E89401400302084B780102084BE8F437
:10083F002401254CF8400302084B78FF88242278C6
:10084F00FFC26420693D206A12D264C3E541940A55
:10085F004009C3E52594405002C26479A1E76023A3
:0D086F00E541601F74FF8541F0848539F07C
:10087C00306A0375F005A4F8C5F0600278FFC3E890
:10088C0095675002A867886622C3E5409440E5410D
:10089C009401E56650031401A6046002F566227803
:1008AC0083E6F520120F4475E89012055375E89015
:1008BC00E5E820ECFBA8BDA9BE120FDE75715575DD
:1008CC007200C3740013FD7455606613FC74552CD0
:1008DC00FC74003DFDECFAEDFBC3E89AE99B401477
:1008EC00E5712455F571E5723400F572EA2CFAEBDA
:1008FC003DFB80E5AE71AF72C3E57213F9E5711380
:10090C00F8C3E913F9E813F87A03C3E913F9E81308
:10091C00F8DAF7AA201A70097571007572000209CD
:10092C003D1AEA6008EE28FEEF39FFDAF88E718F77
:10093C00722275E890227883E6FFE5E820ECF7A8B0
:10094C00BDA9BE0573C3E57394084052757300E9E5
:10095C00FA79A0E76044EA7007E574601B02097835
:10096C00C3E895746010E5745006600C1402098499
:10097C000460F9020984E574F574C3946D401B7529
:10098C0064C0C394044013756480C39404400B7515
:10099C006440C39404400375640075BB0822EFC324
:1009AC009401601F7455601BC3E894FFE9940350D5
:1009BC0012C3E89571E995725009E564600C1564F1
:1009CC000209D6E564F460020564A864C3E52498C2
:1009DC005002A824C3E89565400AA865E565F46053
:1009EC000385656488258826E573B4070375BB10F9
:1009FC0022743279A687F0A4C5F0A2F733F8C3E8C5
:100A0C0095644002A86488228824882588268867F3
:100A1C00227540007541F022C2AF75C820A8CCA940
:100A2C00CDAA3A30CF010A75C824D2AFAB3BAC3C4F
:100A3C00883B893CC3E89BF8E99C206908F930673E
:100A4C000261394196AD3D8A3DF9EA9DFA60047820
:100A5C00FF79FFAE3EAF3F8B3E8C3FC3EC9FFCC398
:100A6C00E99CF542A83BA93CC3E89EF8E99FF9C371
:100A7C00E54113FBE54013FAE82AF540E93BF54163
:100A8C0050067540FF7541FF41E0AA40AB41AC40B8
:100A9C00AD417E047F02C3EB940440021E1FC3EBE6
:100AAC00940840021E1FC3ED13FDEC13FCDEF7C3CC
:100ABC00EA9CFAEB9DFBEF6009C3E913F9E813F824
:100ACC00DFF7EA28FAEB39FB8A408B4150067BFFB3
:100ADC008B408B41C3EB94025002D2673069047F88
:100AEC0003610B7892E6FFC3E537948240110FC384
:100AFC00E53794A040010FC3EF940640027F057EBA
:100B0C0006E541C4540FF9E541C454F0F8E540C47E
:100B1C00540F28F8C3E89EFAE99400FB4009C3EA95
:100B2C009402EB940050047A02E4FB6185AA40AB7A
:100B3C0041EBC4FEEAC4540F4EFCC3EA9CFAEB949E
:100B4C0000FBC3E813C313F8EA28FAEB3400FB8A62
:100B5C00408B41C3EB94024002C2677806EBC4FEA3
:100B6C007B00EAC4540F4EFAC3EA98FA4005C394CA
:100B7C000250027A027892E6FF306002618585525B
:100B8C0056855357D26043E680C3E49AF8E49BF948
:100B9C00306702811FE8FAE9FBD3E913FDE813FC87
:100BAC0088528953C3EF94036038EF20E00DE82C92
:100BBC00F8E93DF9ECFAEDFB020BDAE828F8E93933
:100BCC00F9C3E82402F8E93400F97AFE7BFFC3EF9D
:100BDC009403400E8A548B55884E894F8C508D51FE
:100BEC008153885489558A4E8B4F8C508D51306966
:100BFC0020C3E53394034019E542A2E713F8E55509
:100C0C00F4240138400B20E7087554FFF42401F557
:100C1C00558153E8FAD3E813FC8852C3EF94036070
:100C2C0020EF20E007E82CF8ECFA813FE8282402BA
:100C3C00F87AFEC3EF940340088A54884E8C508196
:100C4C005388548A4E8C50E56BC3335002646BF559
:100C5C006B306002815D753402D26043E680E52D15
:0F0C6C0054066026A840A941C3E913F9E813F81C
:100C7B00C2AF53E67F759100C3E498F594E499F500
:100C8B0095759104D26043E680D2AF22D26575444C
:100C9B0000752000306B03752040020CB6D26575D1
:100CAB004400752040306B03752000D2AF780120D3
:100CBB006722E52D54066002C265C3E541940540E9
:100CCB0013780294054008780394054002780630A7
:100CDB006902780A206019E544601530690AC3E59A
:100CEB003394034003D53406D2AFD26CA187916500
:100CFB00D2AF0000C2AF206726E541C3FB940F4083
:100D0B00027B0FEB240530730123306A0274282019
:100D1B00620123F93069027982E58BC39940B505ED
:100D2B0044E59B5440B52002A17130690A08C3E821
:100D3B00940A40010881DF20650281B6C26553E643
:100D4B007F7591003067107594007595FE75910451
:100D5B00D26043E68081B6AE40AF41C3E49EF594CA
:100D6B00E49FF595A158C3E5339402500281B63048
:100D7B00650281B6D802A18581DFC26C53E67F750F
:100D8B009100855494855595759104854E56854FE4
:100D9B0057D26043E680D2AFE52D54066008206A37
:100DAB00020533020DC1306C0D206B0A206507154F
:100DBB0081158102161122780030640530650278A6
:100DCB0001E53775F007A4F9E5F028F5F0E9A2F095
:100DDB0013A2F113A2F213F537C3947850037537AE
:100DEB0078C3E53795384008D266C293C297C2954F
:100DFB00306002A1FB855056855157D26043E68087
:100E0B0022207D11C2AF754302C296D292D2AF752A
:100E1B009F11020FDBC2AF754302C296D294D2AFC1
:100E2B00759F11020FDB307243207D20C2AF7543DB
:100E3B000390013D757E40C295C294306204D297F7
:100E4B00C14FD296D2AF759F10020FDBC2AF754365
:100E5B000390013D757E40C293C292306204D297DB
:100E6B00C16FD296D2AF759F13020FDB207D17C2D5
:100E7B00AF754303900118C295306202D297D2AF7F
:100E8B00759F10020FDBC2AF754303900118C2931D
:100E9B00306202D297D2AF759F13020FDB207D1108
:100EAB00C2AF754304C292D294D2AF759F13020F97
:100EBB00DBC2AF754304C294D292D2AF759F1002BE
:100ECB000FDB307243207D20C2AF75430590012CA0
:100EDB00757E04C297C296306204D293C1EBD29254
:100EEB00D2AF759F11020FDBC2AF75430590014E58
:100EFB00757E10C297C296306204D295E10BD294E4
:100F0B00D2AF759F11020FDB207D17C2AF75430562
:100F1B0090010EC297306202D293D2AF759F11022D
:100F2B000FDBC2AF754305900122C2973062EBD243
:100F3B0095D2AF759F11020FDB207D11C2AF7543A8
:100F4B0006C294D296D2AF759F10020FDBC2AF755B
:100F5B004306C292D296D2AF759F13020FDB30724B
:100F6B0042207D20C2AF75430190014E757E10C2A9
:100F7B0093C292306204D295E187D294D2AF759F1F
:100F8B0013020FDBC2AF75430190012C757E04C2B7
:100F9B0095C294306204D293E1A7D292D2AF759FDF
:100FAB0010E1DB207D16C2AF754301900122C29385
:100FBB00306202D295D2AF759F13E1DBC2AF75439E
:100FCB000190010EC295306202D293D2AF759F1081
:100FDB00C2662290010C757E00C293C297C295C265
:100FEB0092C296C294C2622278807607087607086E
:100FFB0076010876040876FF0876FF0876080876EF
:10100B0002087601087601788C760108760008765E
:10101B00B40876FF0876FF0876FF0876030876FF9C
:10102B000876010876FF0876250876D008767808CA
:10103B0076C80876040876FF0876010876000876ED
:10104B007A0876100876010876010876000876FF94
:10105B00227887E6FFC2727888C27DE630E102D241
:0F106B007DC27E7889E630E102D27EC3EF940227
:10107A006008758E01D273021089758E00C27322C0
:10108A007880E6149000809378A4F67881E614902C
:10109A0000809378A5F67886E61490008D9378A65A
:1010AA00F6789FE6F8700108C3E8941140027811B7
:1010BA00E82828F56E256E256E28F56F256E2828F6
:1010CA00F570789CE67538FF75390CB402067538E8
:1010DA00A075390AB4030675388275390578A3E60E
:1010EA001490009A93F569120FDE22227896E6FA96
:1010FA007897E6FB7888E6B40305C3EB940EFB30D9
:10110A007F047A007BFFC3EB9AFCC3948250027C73
:10111A00827575000575EC8575F0A4C3E5F0947DBC
:10112A0040F222D27F11F61205627A007B007C100F
:10113A00120558E55F2AFA74003BFBDCF37C04C312
:10114A00EB13FBEA13FADCF7FEC27F11F622E5EF96
:10115A0020E6037520000520903FFFE52014600675
:10116A00901DFF1460009304600375EF1253D9BFFA
:10117A007581C043FF8012055375EF0243B203E540
:10118A00B3240420E70DF521E5E320E0068521B329
:10119A0043E301120FDE7580FF75A40075F1B27585
:1011AA00D4DF75900375A5FC75F2FC75D50375A699
:1011BA000175E241E4F8F6D8FD756B01120FF312DE
:1011CA00165978988676753001C2AF12056C1205E9
:1011DA007C12056212058312056212058A120562E3
:1011EA0012177C12056C12056C120567C2AF78FAE9
:1011FA0079FA308507D9FBD8F7021C00115C118AED
:10120A0011F511F678988676120FDE758850758971
:10121A001275C82475910475D84075A82275B8024C
:10122A0075E690759B80759D0075D10E75BC5875D5
:10123A00BB0875BA1175E880120553D2AF1208AB14
:10124A0053DACF207E0343DA20307E0343DA104399
:10125A00DA01C2D8C27112056CD2617B037A0CE53D
:10126A005E70077A0CDB030211F612056220700326
:10127A000211F6C270E55FC3940240E1E52F541FE4
:10128A00856160F561B560D5DAD5C26153DACF20E0
:10129A007E0343DA20307E0343DA10C2D8C2717863
:1012AA00A2E67008D274E52F54E0F52FC2757529AD
:1012BA0000120567307409C3E529940A4002D27501
:1012CA0012055878023074027800C3E55F9840F03E
:1012DA00C2AF12057C12057C12057CD2AF12056CD6
:1012EA00754D00120558788CE6C394015003021319
:1012FA00C3E530C3940150030213C3207435C3E518
:10130A005F94FF50030213C3C2AF120591D2AF120A
:10131A000567C3E55F940150EFC2AF12057C120561
:10132A005D12057CD2AF120567C3E55F94FF40E901
:10133A000218017F05D27F11F6120567C2AFC27F7C
:10134A0011F6AE5FC3E55F947FD2AF4076120553C4
:10135A00C2AF120591D2AFDFDC312DC3EE9405780E
:10136A0097F612056C12169B1217847F0AD27F1108
:10137A00F6120567C2AFC27F11F6AE5FC3E55F948E
:10138A007FD2AF50E6120553C2AF12057C12055D3B
:10139A0012057CD2AFDFD6312DEE24057896F612EF
:1013AA00056C12169B1217B312056711F6C3E55F97
:1013BA0094FF50026105021801C3E55F954D400391
:1013CA00855F4D12056778017988E7B403027805CD
:1013DA00C3E55F98400241EDC2AF12059112059133
:1013EA00120591D2AF12056C753000E4F531F53271
:1013FA000531E531F470390532789AE678191460C6
:10140A0012783214600D787D14600878FA1460033B
:10141A00753200C3E53298401715327531B47899A0
:10142A008676C2AF120591D2AF7898867612056792
:10143A0012055DE52A700530740221F678012074E0
:10144A00027806C3E55F9840A7120567E52A70038C
:10145A000211F6C2AF120FDEE4F522F523F524F5E8
:0F146A0025F526F56AD2AF7885E6C333F568E439
:10147900F545F546F547F548F549F573F52CF52D8C
:10148900F53775730875BB1012055312093EE5E867
:1014990020ECFBA8BDA9BEE97001F88874120942C5
:1014A90075730875BB107887E6FE7602115C78873C
:1014B900EEF6C2AF7564FF1209FD852264852265C7
:1014C900852266D2AF75220175240175250175261D
:1014D9000185636C756D017888E6B40307C27D30B8
:1014E9007602D27DD268D269753300120F44120F89
:1014F90069120A1D120A24120A1D120A24120A1D4F
:10150900021518C2AF115CD2AF75730075BB081212
:101519000CA812065C120DC2120E0C120A24120C2F
:1015290097306D031206FC20670312084E306703DB
:10153900120895120DC2120E31120A24120CA8308B
:101549006D03120738120DC2120EA8120A24120CCA
:1015590097306D03120796120DC2120ECD120A248E
:10156900120CA8306D031207F3120DC2120F4412A8
:101579000A2412093E120C97120DC2120F691209A0
:1015890042120A2430692F206B2C856764856765B0
:1015990085636C756D0179187A0CC3E53399400937
:1015A900C269D26A8A350215BFC3E55F9401400357
:1015B900021518021619306A1B206B18E5351470CC
:1015C90004C26AA10CF535C3E55F94014003021515
:1015D90018021619753600C3E5629401400985673A
:1015E9006585636C756D01C3E56278FA98502130A1
:1015F9007404E52A601A78F0306B058567647820F1
:10160900C3E541985002A1180536E55F6002C11C87
:10161900753600C2AF120FDE7887E6FE7602115CDE
:101629007887EEF6E4F522F523F524F525F526F578
:1016390068C268D2AF120553120FDE307406E52A6C
:10164900700221F6788DE6C39401400241CA61F522
:10165900901A0D78201216DDE520B4A50CA31216F8
:10166900DDE520B45A0302167B120FF312169B0212
:10167900169A901A0378807B0A1216DDA308DBF903
:10168900901A0F788C7B181216DDA308DBF9901AD3
:101699002722C2AF12171C1216F6901A00740E12E6
:1016A90016E2A374041216E2A374141216E2901A35
:1016B9000378807B0A1216E1A308DBF9901A0F78E8
:1016C9008C7B181216E1A308DBF912172F12170DDC
:1016D900901A2722E493F622E6438F01538FFD7572
:1016E900EF0275B7A575B7F1F0538FFE22438F024C
:1016F900438F0175EF0275B7A575B7F1901A0DF013
:10170900538FFC22901A0D74A5D1E2901A0E745AC7
:10171900D1E2227A3079D07820901A40D1DDE520C3
:10172900F709A3DAF7227A3079D0901A40E7D1E2A3
:1017390009A3DAF922AB77A878BB01027980BB0249
:10174900027981BB03027982BB04027994BB050249
:101759007983BB06027986BB07027992BB080279B5
:1017690087BB0902799CBB0A027988BB0B0279897C
:10177900E8F7227C0512056CDCFB22C2AF12057C5E
:1017890012058312058A12059112055D12057C1254
:10179900058312058A12059112055D12057C120551
:1017A9008312058A120591D2AF22C2AF1205911296
:1017B900058A12058312057C12055D120591120531
:1017C9008A12058312057C12055D12059112058A9C
:1017D90012058312057CD2AF22AE77AF78C2AF1261
:1017E900057C12057C12057C12055DDEF21205915D
:1017F90012055DDFF8D2AF2212178412177C121777
:101809007C7577017578017579001217E27C05AD51
:101819005F12056CC3ED955F70F5C3E55F940140F8
:101829000AC3E55F94FF403702184512173E1216A6
:101839009B121784C2AF75EF1212177CDCD10579A0
:10184900C3E5799403500280C112177C0578E577C6
:101859001490009F93F808C3E57898500280A81265
:0E186900177C12177C0577C3E577940C5002AC
:101877008094120FF312169BC2AF75EF1212177CEA
:0319FD000211587C
:101A00000E041407070104FFFF08020101A55A0193
:101A100000B4FFFFFF03FF01FF25D078C804FF01DA
:081A200000FF10010100FFFFAF
:101A4000235475726E696779363041232020202037
:101A500023424C48454C4923463333302320202031
:101A60002020202020202020202020202020202076
:101C0000C2AFC2D353D9BF7581C043B20343FF8073
:101C1000752438752503B1C975EF0275E24043F1AB
:101C20002053A4DF75D400D2857DFA780379E67C51
:101C300010752200752300901DD67B0675249875BB
:101C400025013085028142208508D8FBD9F9DCF7CF
:101C500081B4308508D8FBD9F9DCF781B4B189E4C7
:101C600093A3C39A6004DDC381B4DBDBB17B600264
:101C7000812B7B08E493FAA3B15CDBF87A30B15C8A
:101C8000752200752300B17BEAFCEBFDC3ED94FEE9
:101C9000400EB17B8A278B28ED30E0048A828B834B
:101CA000B17B7AC270D8C3ED94FE601350CEBD00F4
:101CB00025EC60097520007521FF0200008100A855
:101CC00027A9280809D804D90281D3B17FEA89AAB3
:101CD000F281C50D81A0C3ED94035049EDA2E092BD
:101CE000007AC5C3E5829400E583941C50902000DF
:101CF00010438F02438F0175B7A575B7F1F030001F
:101D00001FA827A9280809438F01538FFDD804D99C
:101D100002A12089AAE275B7A575B7F1F0A3A10DBC
:101D2000538FFC817C7AC1BD030CE493A3FAB140CC
:101D3000DCF8B138817C817EAA22AB23B15CEBFA5E
:101D4000EA6222752608C3E52313F523E52213F57D
:101D50002250066323A0632201D526EAB1C9B1C986
:101D600075260AEAF4200102D285300102C285B14B
:101D7000C9C3134002C201D526EB22B17FEAFB2082
:101D80008502A17F308502A184752608AE24AF2587
:101D9000C3EF13FFEE13FEB1CDB1C9C3EA13308513
:101DA000024480FA30E703632201C3E52313F523DD
:101DB000E52213F52250066323A0632201D526D91C
:101DC000E52265236523F52222AE24AF250E0FDE22
:101DD000FEDFFCD20122424C48656C693437316326
:041DE000F3300601D5
:00000001FF
